:0200000480007A
:10000000B72F0000938F0F8073900F3015A8130047
:100010000000130000001300000013000000130094
:100020000000130000001300000013000000130084
:100030000000130000001300000013000000010086
:10004000970200009382020C73905230814001416C
:100050008141014281420143814301448144014580
:100060008145014681460147814701488148014950
:100070008149014A814A014B814B014C814C014D20
:10008000814D014E814E014F814F971102009381A6
:10009000A1B6170502001305E53A9795030093856D
:1000A000256D014611221705020013052534970519
:1000B0000200938525340146C52817A503001305C2
:1000C000656B97B503009385A56A37B6ABAB13068E
:1000D000B6BAD92817B103001301C169EF40407DBA
:1000E000860293D21200F512638802008242110147
:1000F0006F00001073002030824211017300203025
:10010000711116C0F3222034E3CC02FC82421101AB
:10011000130141F806C20AC40EC612C816CA1ACC88
:100120001ECE22D026D22AD42ED632D836DA3ADCC7
:100130003EDEC2C0C6C2CAC4CEC6D2C8D6CADACC97
:10014000DECEE2D0E6D2EAD4EED6F2D8F6DAFADCA7
:10015000FEDE73252034F32510340A8601A07310C7
:10016000153492402241B2414242D2426243F243AC
:10017000025492542255B2554256D2566257F25703
:10018000064896482649B649464AD64A664BF64B33
:10019000065C965C265DB65D465ED65E665FF65F83
:1001A0001301C1077300203010C16374B50011053D
:1001B000E5BF828000000000000000000000000099
:1001C000000000000000000000000000000000002F
:1001D000000000000000000000000000000000001F
:1001E000000000000000000000000000000000000F
:1001F000197106C00AC20EC412C616C81ACA1ECC8D
:1002000022CE26D02AD22ED432D636D83ADA3EDCC6
:1002100042DEC6C0CAC2CEC4D2C6D6C8DACADECC96
:10022000E2CEE6D0EAD2EED4F2D6F6D8FADAFEDCA6
:100230009702020083A2821B23A02200F322103423
:1002400096DEEF006030170102000321211A0241FF
:10025000F65273901234B72200009382028873A082
:10026000023082403242C2425243E24372448254DC
:100270001255A2553256C2565257E2577258864806
:100280001649A649364AC64A564BE64B764C865C1A
:10029000165DA65D365EC65E565FE65F0961730059
:1002A0002030970202009382E21923A0120023A2B9
:1002B000220023A4320023A6420023A8520023AA2E
:1002C000620023AC720023AE820023A0920223A21C
:1002D000A20223A4B20223A6C20223A8D20223AA06
:1002E000E20223ACF20223AE020323A0120523A2F2
:1002F000220523A4320523A6420523A8520523AADA
:10030000620523AC720523AE820523A0920723A2C7
:10031000A20723A4B20723A6C20723A8D20723AAB1
:10032000E20723ACF207EF40804D170102000321E2
:10033000E10B0241F65273901234B722000093820F
:10034000028873A0023082403242C2425243E243EA
:10035000724482541255A2553256C2565257E25731
:10036000725886481649A649364AC64A564BE64B45
:10037000764C865C165DA65D365EC65E565FE65FB1
:10038000096173002030970202009382A20B83A0C0
:10039000020003A1420083A1820003A2C20083A243
:1003A000020103A3420183A3820103A4C20183A427
:1003B000020203A5420283A5820203A6C20283A60B
:1003C000020303A7420383A7820303A8C20383A8EF
:1003D000020403A9420483A9820403AAC20483AAD3
:1003E000020503AB420583AB820503ACC20583ACB7
:1003F000020603AD420683AD820603AEC20683AE9B
:10040000020703AFC20983AF820782807370043092
:10041000197106C00AC20EC412C616C81ACA1ECC6A
:1004200022CE26D02AD22ED432D636D83ADA3EDCA4
:1004300042DEC6C0CAC2CEC4D2C6D6C8DACADECC74
:10044000E2CEE6D0EAD2EED4F2D6F6D8FADAFEDC84
:100450009702020083A282F923A0220086DEEF1019
:10046000B04017010200032161F80241F652739077
:100470001234B72200009382028873A002308240B7
:100480003242C2425243E243724482541255A25550
:100490003256C2565257E257725886481649A649F4
:1004A000364AC64A564BE64B764C865C165DA65DD0
:1004B000365EC65E565FE65F0961730020309707BF
:1004C0000200938767F39843FD576305F700737045
:1004D000043001A07370043001A041112AC6B24754
:1004E000739047300100410182804111F327403071
:1004F0003EC673F04330B2473E85410182804111D0
:100500002AC62EC432C2B247F1173EC62247B247AE
:1005100098C3B247938787FA3EC61247B24798C33B
:10052000B247A1173EC68E873E87B24798C3B247EF
:10053000D1173EC6170700001307A7F8B24798C3A4
:10054000B2473E8541018280411106C6EF40A0239B
:10055000EF10D014AA8799C3EF1010310100B240F8
:100560004101828041112AC6B24713878700B247F2
:10057000D8C3B2477D5798C7B24713878700B247A1
:10058000D8C7B24713878700B24798CBB24723A09A
:10059000070001004101828041112AC6B24723A809
:1005A000070001004101828001112AC62EC4B24712
:1005B000DC433ECEA2477247D8C3F2479847A247D2
:1005C00098C7F2479C472247D8C3F247224798C7AB
:1005D000A247324798CBB2479C4313871700B247D4
:1005E00098C301000561828001112AC62EC4A2476A
:1005F0009C433ECC6247FD576316F700B2479C4BC5
:100600003ECE31A8B247A1073ECE21A0F247DC433F
:100610003ECEF247DC439C436247E379F7FEF24764
:10062000D843A247D8C3A247DC43224798C7A24772
:10063000724798C7F2472247D8C3A247324798CBA0
:10064000B2479C4313871700B24798C30100056166
:10065000828001112AC6B2479C4B3ECEB247DC4392
:100660003247184798C7B2479C4732475843D8C3C8
:10067000F247DC4332476316F700B2479847F24728
:10068000D8C3B24723A80700F2479C431387F7FF5C
:10069000F24798C3F2479C433E8505618280797199
:1006A00006D622D42AC62EC4B2473ECEF24781E7F0
:1006B0007370043001A0EF202057F2478043F247C7
:1006C000D85FF247BC43BE853A85EF50A02AAA877F
:1006D0003307F400F247D8C3F24723AC0702F247CE
:1006E0009843F24798C7F2478043F247DC5F13878D
:1006F000F7FFF247BC43BE853A85EF50A027AA8793
:100700003307F400F247D8C7F2477D57F8C3F247E2
:100710007D57B8C7A24799EFF2479C4B8DC7F24768
:10072000C1073E85EF1090402A878547631DF7007B
:10073000F13911A8F247C1073E852D35F24793875D
:1007400047023E850535EF20005185473E85B25072
:10075000225445618280797106D62AC62EC4B2879A
:10076000A303F10002CCB24781E77370043001A00B
:10077000A24799E302CE01A8A2453245EF50801F5F
:10078000AA8785073ECEF247938747053E85EF301F
:10079000805C2ACAD24785CFA24789E7D247524711
:1007A00098C331A0D24713874705D24798C3D24791
:1007B0003247D8DFD2472247B8C385455245C535B1
:1007C000D247034771002388E704D2473ECCE24773
:1007D00081E77370043001A0E2473E85B250456165
:1007E0008280797106D6AA87A307F1001305400518
:1007F000EF3060562ACEF247B9CFF24723A2070066
:10080000F24723A00700F24723A40700F24723A6DC
:100810000700F24723AC0702F2470547D8DFF2474B
:1008200023A00704F2477D57F8C3F2477D57B8C7A6
:10083000F2470347F1002388E704F247C1073E85EA
:100840001533F247938747023E85293B814601468F
:10085000814572453122F2473E85B2504561828022
:10086000797106D622D42AC6B2473ECCE24781E748
:100870007370043001A0E247C043EF20001DAA8737
:100880006313F402E247DC471387F7FFE247D8C758
:10089000E247DC4791E78146014681456245C92030
:1008A00085473ECE11A002CEF2473E85B25022547B
:1008B00045618280797106D622D42AC62EC4B247F9
:1008C0003ECCE24781E77370043001A0E247C043A9
:1008D000EF20A017AA87631BF400E247DC471387C9
:1008E0001700E247D8C785473ECE0DA08146224675
:1008F00081456245252E2ACE724785476318F70049
:10090000E247DC4713871700E247D8C7F2473E8526
:10091000B250225445618280797106D62AC62EC40F
:10092000B24781E77370043001A02247B24763F5F4
:10093000E7007370043001A0094681453245213D2E
:100940002ACEF24781C7F247224798DFF24781E774
:100950007370043001A0F2473E85B2504561828039
:10096000397106DE2AC62EC432C236C002D6B2475C
:100970003ED4A25781E77370043001A0A24781E7FB
:10098000A257BC4399E3854711A0814781E7737063
:10099000043001A0024789476317F700A257D85FC8
:1009A00085476314F700854711A0814781E773707D
:1009B000043001A0EF20C00AAA8799E3924799E387
:1009C000854711A0814781E77370043001A0EF20B3
:1009D000A025A257985FA257DC5F6366F700024725
:1009E0008947631DF7020246A245225565232AD294
:1009F000A257DC5389CFA257938747023E85EF1059
:100A0000F0122A8785476317F700093421A092570F
:100A100091C3ED3AEF202024854771A8924789E7DA
:100A2000EF206023814741A8B25799E77C083E85B3
:100A3000EF10702785473ED6EF20E021EF10401AD7
:100A4000EF20801EA257F843FD576315F700A25709
:100A500023A20704A257B847FD576315F700A25712
:100A600023A40704EF20201F58007C08BA853E8588
:100A7000EF107026AA879DEB2255EF006071AA87C0
:100A80008DC3A257C1071247BA853E85EF10E070AB
:100A900022551525EF108016AA87E39A07F2BD327A
:100AA0003DB72255092DEF10601515B722552125A8
:100AB000EF10C01481473E85F25021618280797128
:100AC00006D62AC62EC432C236C0B2473ECCE24752
:100AD00081E77370043001A0A24781E7E247BC437D
:100AE00099E3854711A0814781E77370043001A025
:100AF000024789476317F700E247D85F85476314C9
:100B0000F700854711A0814781E77370043001A089
:100B1000E93AAA873ECAE247985FE247DC5F63662C
:100B2000F700024789476315F7040246A24562456C
:100B30009521E247B847FD576313F702E247DC53BC
:100B40008DC7E247938747023E85EF10207EAA8734
:100B500089CF924799CB9247054798C339A0E2477E
:100B6000BC4713871700E247B8C785473ECE11A0A0
:100B700002CED2473E859532F2473E85B25045615E
:100B80008280797106D62AC62EC4B2473ECCE2478F
:100B900081E77370043001A0E247BC4381C77370E2
:100BA000043001A0E2479C4381E7E247DC4399E33C
:100BB000854711A0814781E77370043001A0353269
:100BC000AA873ECAE247985FE247DC5F6377F70493
:100BD000E2479C5F13871700E24798DFE247B84778
:100BE000FD576313F702E247DC538DC7E247938753
:100BF00047023E85EF108073AA8789CFA24799CB21
:100C0000A247054798C339A0E247BC47138717009E
:100C1000E247B8C785473ECE11A002CED2473E85F7
:100C20006D38F2473E85B25045618280397106DEEB
:100C30002AC62EC432C236C002D6B2473ED4A2570C
:100C400081E77370043001A0A24781E7A257BC433B
:100C500099E3854711A0814781E77370043001A0B3
:100C6000EF101060AA8799E3924799E3854711A096
:100C7000814781E77370043001A0EF10F07AA2572A
:100C80009C5FB5CBA257DC473ED2A2452255F92E38
:100C9000824795EFA2579C5F1387F7FFA25798DF13
:100CA000A2579C4391E7EF2060022A87A257D8C33E
:100CB000A2579C4B8DCFA257C1073E85EF1000670E
:100CC0002A8785476315F702EFF04FF40DA0A2576E
:100CD0001257D8C7A257DC5399CBA2579387470224
:100CE0003E85EF10A064AA8799C3EFF02FF2EF10B2
:100CF000907685475DA8924789E7EF10D0758147C8
:100D00006DA0B25799E77C083E85EF10C079854702
:100D10003ED6EF105074EF00B06CEF10F070A25799
:100D2000F843FD576315F700A25723A20704A25703
:100D3000B847FD576315F700A25723A40704EF1027
:100D4000907158007C08BA853E85EF10C078AA875C
:100D5000A1EB2255CD2EAA879DCFA2579C4391EBA4
:100D6000EF10906CA257DC433E85EF107052EF10ED
:100D7000906EA257938747021247BA853E85EF10BF
:100D8000C04122550D2EEF007067AA87E39707EE4A
:100D9000EFF0CFE7DDB52255392EEF003066F1BD1B
:100DA0002255112EEF00906581473E85F25021615A
:100DB0008280797106D62AC62EC432C2B2473ECC92
:100DC000E24781E77370043001A0A24781E7E24760
:100DD000BC4399E3854711A0814781E773700430D4
:100DE00001A0EFF08FF0AA873ECAE2479C5FA1CB3B
:100DF000A2456245A52CE2479C5F1387F7FFE247B7
:100E000098DFE247F843FD576312F702E2479C4B35
:100E100085C7E247C1073E85EF104051AA8789CFB9
:100E2000924799CB9247054798C339A0E247FC43C4
:100E300013871700E247F8C385473ECE11A002CEC4
:100E4000D2473E85EFF06FE9F2473E85B2504561EB
:100E50008280797106D62AC62EC4B2473ECCE247BC
:100E600081E77370043001A0A24781E7E247BC43E9
:100E700099E3854711A0814781E77370043001A091
:100E8000E247BC4381E77370043001A0EFF0EFE567
:100E9000AA873ECAE2479C5F89CFE247DC473EC84B
:100EA000A2456245E122E2474247D8C785473ECE88
:100EB00011A002CED2473E85EFF02FE2F2473E85E9
:100EC000B25045618280797106D62AC6B24781E761
:100ED0007370043001A0EF103055B2479C5F3ECED6
:100EE000EF107057F2473E85B250456182807971AC
:100EF00006D62AC6B2473ECEF24781E77370043069
:100F000001A0EF107052F247D85FF2479C5FB30721
:100F1000F7403ECCEF103054E2473E85B250456179
:100F2000828001112AC6B24781E77370043001A0A4
:100F3000B2479C5F3ECEF2473E8505618280797163
:100F400006D62AC6B2473ECEF24781E77370043018
:100F500001A07245E5247245EF20F0720100B25005
:100F60004561828041112AC6B247FC473E85410156
:100F7000828041112AC62EC4B2472247F8C7010019
:100F80004101828041112AC6B24783C707053E85C9
:100F900041018280797106D62AC62EC432C202CEA1
:100FA000B247BC4391EFB2479C43D5E7B247DC431D
:100FB0003E85EF10903B2ACEB24723A2070061A8DE
:100FC000924785EFB2479847B247BC433E86A24559
:100FD0003A85EF20F079B2479847B247BC433E9735
:100FE000B24798C7B2479847B247DC436365F706F4
:100FF000B2479843B24798C7B9A8B247D847B24753
:10100000BC433E86A2453A85EF209076B247D8474A
:10101000B247BC43B307F0403E97B247D8C7B24788
:10102000D847B2479C43637BF700B247D843B247E7
:10103000BC43B307F0403E97B247D8C71247894731
:10104000631BF700B2479C5F99C7B2479C5F138749
:10105000F7FFB24798DFB2479C5F13871700B2478C
:1010600098DFF2473E85B25045618280011106CE7D
:101070002AC62EC4B247BC439DCBB247D847B2471D
:10108000BC433E97B247D8C7B247D847B247DC43C4
:101090006366F700B2479843B247D8C7B247D8470C
:1010A000B247BC433E86BA852245EF20706C0100F2
:1010B000F24005618280011106CE2AC6EF10D036BB
:1010C00025A0B247DC5395C7B247938747023E85B8
:1010D000EF10C025AA8799C3EF104049B247BC471B
:1010E0001387F7FFB247B8C7B247BC47E34BF0FCE2
:1010F00011A00100B2477D57B8C7EF10D035EF10EF
:10110000B0321DA0B2479C4B8DC7B247C1073E8588
:10111000EF10C021AA8799C3EF104045B247FC43A6
:101120001387F7FFB247F8C3B247FC43E34CF0FC28
:1011300011A00100B2477D57F8C3EF10D031010074
:10114000F24005618280797106D62AC6EF10D02D53
:10115000B2479C5F81E785473ECE11A002CEEF10DB
:10116000902FF2473E85B2504561828001112AC618
:10117000B24781E77370043001A0B2479C5F81E7FA
:1011800085473ECE11A002CEF2473E8505618280A2
:10119000797106D62AC6EF103029B247985FB24758
:1011A000DC5F6315F70085473ECE11A002CEEF103D
:1011B000902AF2473E85B2504561828001112AC6CD
:1011C000B24781E77370043001A0B247985FB2471D
:1011D000DC5F6315F70085473ECE11A002CEF247D3
:1011E0003E850561828001112AC62EC402CE81A0EF
:1011F0001787030013070754F2478E07BA979C43DB
:1012000085E7178703001307E752F2478E07BA975F
:10121000224798C3178703001307C751F2478E0769
:10122000BA973247D8C301A8F24785073ECE724726
:101230009D47E3FFE7FA01000561828001112AC69C
:1012400002CE0DA8178703001307C74EF2478E077B
:10125000BA97DC433247631CF70017870300130774
:10126000674DF2478E07BA9723A0070001A8F247FF
:1012700085073ECE72479D47E3F6E7FC0100056116
:101280008280797106D62AC62EC432C2B2473ECEBB
:10129000EF109019F247F843FD576315F700F24736
:1012A00023A20704F247B847FD576315F700F2473A
:1012B00023A40704EF10301AF2479C5F89EBF24732
:1012C000938747021246A2453E85EF00907E724505
:1012D000DD330100B25045618280397106DE2ACECD
:1012E0002ECC36C83AC63EC442C246C0B287231B83
:1012F000F100F24781E77370043001A03247A5473F
:1013000063F5E7007370043001A0835761019245D3
:101310003E85EF1080512AD4A257638F0712A2573F
:10132000985B83566101B7070040FD17B6978A079F
:10133000BA973ED29257F19B3ED292578D8B81C77E
:101340007370043001A0835761013E8782463246A4
:10135000E2452255EF10E0274246F2451255EFF0E4
:101360000F9A2A87A25798C3A24781C7A24722573C
:1013700098C3EF10700B97F701009387E7279C4302
:101380001387170097F701009387072798C397F7EC
:1013900001009387A7059C4395E397F70100938786
:1013A000E704225798C397F701009387E7249843EF
:1013B0008547631AF702EF10C02C35A097F701009C
:1013C000938747249C4385E397F70100938707029F
:1013D0009C43DC5732476368F70097F70100938717
:1013E000E700225798C397F701009387A7229C43F1
:1013F0001387170097F701009387C72198C397F7C2
:101400000100938727219843A257B8C7A257D857FE
:1014100097F701009387C71E9C4363F9E700A25723
:10142000D85797F701009387A71D98C3A257D8579D
:10143000BA878A07BA978A0717F701001307470880
:101440003E97A2579107BE853A85EFF0EF95854705
:101450003ED6EF10500019A0FD573ED632578547B3
:101460006313F70297F701009387C7199C4381CF55
:1014700097F70100938787F79C43DC57324763F463
:10148000E700EFE0BFF8B2573E85F250216182805D
:10149000797106D62AC6EF102079B24799E797F7F7
:1014A00001009387A7F49C4311A0B2473ECEF247B8
:1014B00091073E85EFF0EF99F2479C5791C7F247AD
:1014C000E1073E85EFF0EF98F2479107BE8517F5EB
:1014D00001001305A50FEFF02F8D97F701009387FB
:1014E00027109C431387170097F701009387470F36
:1014F00098C397F701009387E7119C431387170060
:1015000097F701009387071198C3EF10C07497F7FE
:1015100001009387270F9C439DCB97F7010093878A
:10152000E7EC9C437247631EF70097F7010093872F
:10153000E70E9C4381C77370043001A0EFE01FEDFC
:1015400039A0EF10606EEF10A04BEF10C0700100DB
:10155000B25045618280797106D62AC62EC402CE69
:10156000B24781E77370043001A0A24781E773702E
:10157000043001A097F701009387470A9C4381C775
:101580007370043001A0A92D97F701009387070716
:101590009C433ECCB2479C432247BA973ECAB247CF
:1015A0009C436247637EF700B2479C435247637493
:1015B000F7025247E24763F0E70285473ECE21A893
:1015C000B2479C4352476366F7005247E24763F4D1
:1015D000E70085473ECEB247524798C3F24789CFCE
:1015E00097F70100938787E09C4391073E85EFF0D2
:1015F0004F865245EF10001B11252AC8C24799E3B8
:10160000EFE0DFE00100B25045618280797106D6DB
:101610002AC602CEB247A9C397F7010093870700F5
:101620009C4381C77370043001A05D2B97F70100C4
:101630009387C7FC9C433247BA973ECC97F701008B
:101640009387C7DA9C4391073E85EFF08F80624510
:10165000EF10401565232ACEF24799E3EFE01FDB38
:101660000100B25045618280797106D62AC6B24720
:101670003ECCE24781E77370043001A097F7010088
:101680009387C7D69C4362476314F70002CEBDA080
:10169000EF108059E247DC4B3ECAEF10C05B97F772
:1016A00001009387E7F09C435247630AF70097F7DE
:1016B0000100938727F09C4352476315F700894741
:1016C0003ECE2DA8524797F701009387A7F1631BE1
:1016D000F700E2479C5781E78D473ECE05A089473A
:1016E0003ECE29A8524797F70100938727EE63154E
:1016F000F70091473ECE19A085473ECEF2473E8582
:10170000B25045618280797106D62AC6EF10C05169
:10171000B24799E797F70100938747CD9C4311A003
:10172000B2473ECEF247DC573ECCEF10C052E24704
:101730003E85B25045618280797106D62AC6EFE0B7
:10174000DFDAAA873ECEB24799E797F70100938781
:10175000E7C99C4311A0B2473ECCE247DC573ECAE2
:10176000F2473E85EFE07FD7D2473E85B2504561D4
:101770008280797106D62AC62EC402CE2247A5479A
:1017800063F5E7007370043001A02247A54763F4B6
:10179000E700A5473EC4EF102049B24799E797F705
:1017A00001009387A7C49C4311A0B2473ECCE247F7
:1017B000BC4B3ECA5247A247630AF70E2247D247A4
:1017C00063F6E70297F70100938747C29C4362479D
:1017D0006308F70297F70100938747C19C43DC57E2
:1017E0002247636FF70085473ECE19A897F701009F
:1017F0009387C7BF9C4362476314F70085473ECE7B
:10180000E247DC573EC8E247B84BE247DC57631576
:10181000F700E2472247D8D7E2472247B8CBE24752
:101820009C4F63C707002947A2471D8FE24798CF07
:10183000E247D44B4247BA878A07BA978A0717F715
:1018400001001307E7C7BA976394F600854711A014
:101850008147B9C7E24791073E85EFE09FDFE24746
:10186000D85797F701009387A7D99C4363F9E700FE
:10187000E247D85797F70100938787D898C3E24784
:10188000D857BA878A07BA978A0717F7010013074C
:1018900027C33E97E2479107BE853A85EFE0DFD048
:1018A000724785476314F700EFE05FB6EF10A03A88
:1018B0000100B25045618280797106D62AC6EF10C8
:1018C000A036B24799E797F70100938727B29C4368
:1018D00011A0B2473ECEF24791073E85EFE07FD799
:1018E000F2479C5791C7F247E1073E85EFE07FD66C
:1018F000F2479107BE8517F501001305A5CEEFE06D
:10190000BFCAEF10403597F70100938727AE9C437D
:1019100072476319F70497F701009387A7CE9C439A
:1019200089CF97F70100938767CF9C4381C7737076
:10193000043001A0EFE09FAD91A097F701009387DD
:1019400067CA984397F70100938707CB9C436319B5
:10195000F70097F70100938767A923A0070039A82C
:10196000212729A897F701009387C7C99C4399C7E6
:10197000EF10802BEF10C008EF10E02D0100B250E7
:101980004561828001112AC602CEB2473ECCB247E1
:1019900081E77370043001A0E247D84B97F701004C
:1019A000938747C46314F700854711A0814795C307
:1019B000E247985797F70100938707C0630BF7003A
:1019C000E2479C5799E3854711A0814799C3854712
:1019D0003ECEF2473E8505618280797106D62AC6E1
:1019E000B2473ECEB24781E77370043001A0F247A0
:1019F000C9C797F701009387679F9C437247630E9F
:101A0000F706EF1060227245B53F2A8785476314B9
:101A1000F706F24791073E85EFE0BFC3F247D8577C
:101A200097F701009387C7BD9C4363F9E700F2472E
:101A3000D85797F701009387A7BC98C3F247D857A8
:101A4000BA878A07BA978A0717F70100130747A7CB
:101A50003E97F2479107BE853A85EFE0FFB4F24723
:101A6000D85797F70100938767989C43DC576364C6
:101A7000F700EFE0BF99EF10001E0100B250456182
:101A80008280797106D62AC602CEB2473ECCB247D2
:101A900081E77370043001A0EFE03FA5AA873ECA3A
:101AA0006245CD352A8785476314F70897F701000B
:101AB0009387C7B69C43A5E7E247D85797F701003D
:101AC0009387C7929C43DC576364F70085473ECEFB
:101AD000E24791073E85EFE0DFB7E247D85797F737
:101AE00001009387E7B19C4363F9E700E247D857C9
:101AF00097F701009387C7B098C3E247D857BA87D2
:101B00008A07BA978A0717F701001307679B3E9762
:101B1000E2479107BE853A85EFE01FA911A8E24789
:101B2000E107BE8517F50100130505A9EFE0DFA762
:101B3000D2473E85EFE07F9AF2473E85B25045613D
:101B40008280011106CE81480148814701478146C4
:101B50001306004097E501009385C54A171500005C
:101B6000130585A5EFF06FF72AC632478547631541
:101B7000F700EF10C06D2AC6324785476319F70298
:101B80007370043097F70100938707A97D5798C3B6
:101B900097F70100938707A7054798C397F70100B8
:101BA0009387C7A523A00700EFE0AFEF31A0B247AE
:101BB00081E77370043001A00100F240056182806A
:101BC000411106C67370043097F70100938787A30D
:101BD00023A00700EFE02FFB0100B240410182800B
:101BE00097F70100938787A39C431387170097F704
:101BF00001009387A7A298C301008280011106CE3D
:101C000002C697F70100938767A19C4381E7737031
:101C1000043001A0EF10400197F70100938707A05F
:101C20009C431387F7FF97F701009387279F98C37B
:101C300097F701009387879E9C436390071097F75F
:101C400001009387679B9C436389070E59A097F710
:101C5000010093876796DC47DC473EC4A247E10753
:101C60003E85EFE01F9FA24791073E85EFE07F9EF4
:101C7000A247D85797F70100938787989C4363F949
:101C8000E700A247D85797F701009387679798C353
:101C9000A247D857BA878A07BA978A0717F7010069
:101CA000130707823E97A2479107BE853A85EFE06A
:101CB000BF8FA247D85797E70100938727739C43AC
:101CC000DC576368F70097F701009387279405476F
:101CD00098C397F701009387278E9C43ADFB97F736
:101CE0000100938767929C438DCF35A0452AAA8730
:101CF00099C797F7010093876791054798C397F7AE
:101D00000100938767909C431387F7FF97F70100C3
:101D10009387878F98C397F701009387E78E9C433B
:101D2000F1F797F701009387678E9843854763160D
:101D3000F70085473EC6EFE06FEDEF00D071B24788
:101D40003E85F24005618280011106CEEF00D06D24
:101D500097F701009387878A9C433EC6EF00B06FD8
:101D6000B2473E85F24005618280011106CEEFE068
:101D7000CFF7AA873EC697F70100938727889C4331
:101D80003EC4B2473E85EFE04FF5A2473E85F240A4
:101D90000561828097F70100938707869C433E8503
:101DA0008280797106D62AC62EC432C202CEA947D5
:101DB0003ECC3D3597F70100938707849C4322472B
:101DC0006368F70CE247FD173ECCF24796073247AF
:101DD000B306F7006247BA878A07BA978A0717E7F8
:101DE00001001307E76DBA970546BE853685EF00FB
:101DF000902A2A87F247BA973ECEE247E1F7F247A8
:101E0000960732473E9797E701009387677A9C438E
:101E10000946BE853A85EF0010282A87F247BA970F
:101E20003ECEF247960732473E9797E701009387E9
:101E300067789C430946BE853A85EF00D0252A87FE
:101E4000F247BA973ECEF24796073247BA97114605
:101E500097E50100938585773E85EF00D0232A879B
:101E6000F247BA973ECEF24796073247BA970D46E9
:101E700097E50100938505773E85EF00D0212A87FD
:101E8000F247BA973ECE924781C7924723A00700F8
:101E9000B533F2473E85B25045618280797106D6EE
:101EA00002CE97E70100938767779C4363950718F5
:101EB00097E70100938787749C431387170097E780
:101EC00001009387A77398C397E70100938707736F
:101ED0009C433ECCE247B9EF97E701009387476DFB
:101EE0009C439C4381C77370043001A097E70100B5
:101EF0009387076C9C433ECA97E701009387876BE3
:101F0000984397E701009387A76A98C397E7010072
:101F10009387476A524798C397E701009387476FB3
:101F20009C431387170097E701009387676E98C358
:101F3000EF00102D97E701009387076E9C436247DF
:101F40006365F70C97E70100938787669C439C4382
:101F500099E3854711A0814781CB97E701009387DB
:101F6000A76B7D5798C355A097E7010093874764F7
:101F70009C43DC47DC473EC8C247DC433EC6624761
:101F8000B2476379F70097E701009387E768324724
:101F900098C3A5A8C24791073E85EFE08FEBC247E3
:101FA0009C5791C7C247E1073E85EFE08FEAC247E1
:101FB000D85797E701009387A7649C4363F9E7002C
:101FC000C247D85797E701009387876398C3C247F2
:101FD000D857BA878A07BA978A0717E70100130705
:101FE000274E3E97C2479107BE853A85EFE0CFDB8B
:101FF000C247D85797E701009387473F9C43DC5778
:10200000E362F7F485473ECE35BF97E7010093873B
:10201000E73D9C43D85797E601009386664ABA8706
:102020008A07BA978A07B6979843854763F1E7020C
:1020300085473ECE29A897E701009387E75C9C433C
:102040001387170097E701009387075C98C397E70A
:1020500001009387A75B9C4399C385473ECEF24717
:102060003E85B25045618280011106CE97E701009E
:102070009387C75A9C4381CB97E701009387075901
:10208000054798C339A297E701009387275823A0F3
:10209000070097E70100938767359C439C5B3EC62A
:1020A000B7A7A5A59387575A3EC4B2479C4322477A
:1020B0006314F702B24791079C432247631EF7005F
:1020C000B247A1079C4322476318F700B247B10704
:1020D0009C4322476308F70497E701009387073181
:1020E000984397E70100938767309C4393874703A2
:1020F000BE853A85EF20B00A35A097E701009387A7
:1021000027509C4381E77370043001A097E70100DA
:102110009387074F9C431387F7FF97E70100938747
:10212000274E98C397E701009387874D984397E61A
:1021300001009386E638BA878A07BA978A07B69766
:102140009C43C5DF97E701009387874B9843BA8785
:102150008A07BA978A0717E7010013076736BA9705
:102160003EC29247DC43D8439247D8C39247D843F4
:102170009247A1076317F7009247DC43D843924781
:10218000D8C39247DC43D84797E7010093870726D7
:1021900098C30100F24005618280797106D62AC693
:1021A0002EC4B24781E77370043001A097E70100A5
:1021B0009387C7239C43E107BE853245EFE0CFC23A
:1021C00097E70100938787229C4391073E85EFE0C4
:1021D0004FC82247FD576310F70297E70100938726
:1021E000E7209C439107BE8517E501001305853F55
:1021F000EFE08FBB19A897E70100938727409C4326
:102200002247BA973ECE7245712B0100B25045610C
:102210008280797106D62AC62EC432C2B24781E7BF
:102220007370043001A097E701009387273F9C4318
:1022300081E77370043001A097E701009387071BC3
:102240009C43A24637070080558F98CF97E701003F
:102250009387C7199C43E107BE853245EFE0CFB4B1
:1022600097E70100938787189C4391073E85EFE02D
:102270004FBE1247FD576310F70297E7010093879F
:10228000E7169C439107BE8517E5010013058535C8
:10229000EFE08FB119A897E70100938727369C4399
:1022A0001247BA973ECE7245F5290100B2504561FA
:1022B0008280797106D62AC62EC432C2B24781E71F
:1022C0007370043001A097E70100938727129C43A5
:1022D000E107BE853245EFE02FAD97E70100938718
:1022E000E7109C4391073E85EFE0AFB61247854764
:1022F0006310F70297E701009387470F9C4391070C
:10230000BE8517E501001305E52DEFE0EFA919A83B
:1023100097E701009387872E9C432247BA973ECECA
:10232000724549210100B25045618280797106D61B
:102330002AC6B247DC47DC473ECCE24781E77370F0
:10234000043001A0E247E1073E85EFE08FB097E758
:1023500001009387A72C9C43A1EBE24791073E85A0
:10236000EFE02FAFE247D85797E70100938747295F
:102370009C4363F9E700E247D85797E7010093874A
:10238000272898C3E247D857BA878A07BA978A0797
:1023900017E701001307C7123E97E2479107BE8572
:1023A0003A85EFE06FA011A8E247E107BE8517E587
:1023B000010013056520EFE02F9FE247D85797E70C
:1023C00001009387A7029C43DC5763FBE700854726
:1023D0003ECE97E7010093876723054798C311A076
:1023E00002CEF2473E85B25045618280797106D6B1
:1023F0002AC62EC497E70100938747229C4381E7B2
:102400007370043001A02247B70700805D8FB24788
:1024100098C3B247DC473ECCE24781E77370043093
:1024200001A03245EFE0EFA2E24791073E85EFE0E1
:102430004FA2E247D85797E701009387671C9C4358
:1024400063F9E700E247D85797E701009387471BF6
:1024500098C3E247D857BA878A07BA978A0717E717
:1024600001001307E7053E97E2479107BE853A85CD
:10247000EFE08F93E247D85797E70100938707F77C
:102480009C43DC5763FBE70085473ECE97E701009E
:102490009387C717054798C311A002CEF2473E8520
:1024A000B2504561828041112AC6B24781E77370FC
:1024B000043001A097E70100938787159843B2473E
:1024C00098C397E70100938767139843B247D8C32F
:1024D000010041018280797106D62AC62EC4B24716
:1024E00081E77370043001A0A24781E77370043064
:1024F00001A01D2F97E70100938747109C433ECC16
:10250000A2479843FD576314F70002CE91A8B24743
:10251000984397E701009387A70F9C43630AF7004E
:10252000B247DC4362476365F70085473ECE0DA89E
:10253000B247DC4362471D8FA2479C436370F7029A
:10254000A2479843B247D443E247B387F6403E9749
:10255000A24798C33245813F02CE19A085473ECE9F
:10256000DD2DF2473E85B2504561828097E701003C
:102570009387C709054798C30100828001112AC6C5
:10258000B24799C7B2473ECCE247FC473ECE11A0C6
:1025900002CEF2473E850561828001112AC62EC413
:1025A000B24791C7B2473ECEF2472247F8C7010073
:1025B00005618280011106CE2AC6852297E70100B7
:1025C000938707F098438547E3F9E7FEEFD01FE4D0
:1025D000EDB7397106DE2ACE2ECC32CA36C8BA879C
:1025E0002317F10002D625A06247B257BA9703C756
:1025F0000700F246B257B697238AE7026247B257FE
:10260000BA9783C7070089CBB25785073ED63257A2
:10261000BD47E3FBE7FC11A00100F247A3810704DB
:102620005247A54763F4E700A5473ECAF247524721
:10263000D8D7F2475247B8CBF24723AA0704F2474C
:1026400091073E85EFD05FF5F247E1073E85EFD079
:10265000BFF4F247724798CB2947D2471D8FF24704
:1026600098CFF2477247D8D3F24723A20704F24724
:1026700023AC0704F24723AE07040100F2502161A6
:102680008280011106CE02C60DA03247BA878A07A2
:10269000BA978A0717E70100130787E2BA973E85C2
:1026A000EFD05FECB24785073EC63247A547E3FE51
:1026B000E7FC17E50100130525EDEFD0BFEA17E5AC
:1026C00001001305A5EDEFD0FFE917E501001305A3
:1026D000A5EEEFD03FE917E50100130525EFEFD098
:1026E0007FE817E501001305E5EFEFD0BFE797E7B7
:1026F00001009387E7EB17E701001307E7E898C3AA
:1027000097E70100938707EB17E70100130707E935
:1027100098C30100F24005618280011106CE8DA8A8
:10272000EFF00FCC97E70100938747EA9C4393B7FC
:10273000170093F7F70F3EC6EFF04FCCB247A9EB67
:10274000E52197E70100938767E8DC47DC473EC453
:10275000A24791073E85EFD0DFEF97E7010093870F
:10276000A7E99C431387F7FF97E701009387C7E822
:1027700098C397E701009387A7E69C431387F7FF69
:1027800097E701009387C7E598C3F1212245912C73
:1027900097E701009387C7E49C43D9F30100F24017
:1027A00005618280011106CE2AC697E70100938752
:1027B000E7C39C433247D8C397E70100938707E4F8
:1027C0009C4332476372F70297E70100938787DEE5
:1027D000984397E70100938767C19C439107BE85A3
:1027E0003A85EFD07FE035A897E70100938747DC73
:1027F000984397E70100938767BF9C439107BE8585
:102800003A85EFD07FDE97E701009387E7E09C43AE
:1028100032476378F70097E701009387E7DF324795
:1028200098C30100F24005618280797106D6AA87BB
:102830002EC42317F100A24789EB8357E1008A07D2
:102840003E85EF104051AA8711A0A2473ECCE24737
:1028500085C313050006EF1000502ACEF24789C742
:10286000F247624798DB31A06245EF10C06111A0CA
:1028700002CEF24781CFF247985B8357E1008A0787
:102880003E869305500A3A85EF104075F2473E8523
:10289000B25045618280397106DE22DC2AC62EC420
:1028A00032C202D6A2479C43638D070EA2473ED494
:1028B000A257DC43D843A257D8C3A257D843A25744
:1028C000A1076317F700A257DC43D843A257D8C328
:1028D000A257DC43DC473ED2A2473ED08257DC43BE
:1028E000D8438257D8C38257D8438257A10763176A
:1028F000F7008257DC43D8438257D8C38257DC4362
:10290000DC473ECEB25796073247BA97724798C314
:10291000B25796073247BA97724713074703D8C38F
:10292000B25796073247BA977247384798C7B25797
:1029300096073247BA971247D8C7B2579607324719
:10294000BA977247585798CB12478D47631BF700C9
:10295000F2479C5799C7B25796073247BA9709472B
:10296000D8C7B25796073247BA977247384BD8CB79
:10297000B25796073247BA9723AC0700F247945BE9
:10298000B257960732473304F70036850D20AA87E1
:10299000231EF400B25785073ED672479257E31DB7
:1029A000F7F2B2573E85F2506254216182800111E4
:1029B0002AC602CE39A0B24785073EC6F247850730
:1029C0003ECEB24703C707009307500AE305F7FE60
:1029D000F24789833ECEF247C207C1833E85056137
:1029E0008280011106CE2AC6B2479C5B3E85EF105D
:1029F00080493245EF1020490100F2400561828094
:102A0000411197E701009387A7BA9C439C4399E340
:102A1000854711A0814781CB97E701009387C7BF06
:102A20007D5798C305A097E70100938767B89C433B
:102A3000DC47DC473EC6B247D84397E7010093879F
:102A4000A7BD98C3010041018280411197E70100B1
:102A50009387C7999C433EC6B2473E854101828019
:102A6000411197E701009387E7B99C4381E78547C8
:102A70003EC619A897E70100938747BA9C4381E7B0
:102A800089473EC611A002C6B2473E8541018280F9
:102A9000797106D62AC6B2473ECEB247F9C3F2478D
:102AA000D85797E70100938767949C43DC57637A74
:102AB000F70AF2479C4F63CC070097E70100938722
:102AC000E7929C43DC5729471D8FF24798CFF24786
:102AD000D44BF247D857BA878A07BA978A0717E7BD
:102AE00001001307E79DBA976394F600854711A08C
:102AF0008147A5C3F24791073E85EFD09FB597E781
:102B000001009387A78E9C43D857F247D8D7F24746
:102B1000D85797E701009387A7AE9C4363F9E70076
:102B2000F247D85797E70100938787AD98C3F247DC
:102B3000D857BA878A07BA978A0717E70100130799
:102B400027983E97F2479107BE853A85EFD0DFA5DB
:102B500009A897E70100938767899C43D857F247F4
:102B6000D8D70100B25045618280797106D62AC655
:102B7000B2473ECC02CEB247DDC397E70100938750
:102B8000E7869C4362476305F7007370043001A039
:102B9000E247FC4B81E77370043001A0E247FC4B35
:102BA0001387F7FFE247F8CBE247D857E247BC4B21
:102BB0006307F706E247FC4BBDE3E24791073E851A
:102BC000EFD03FA9E247B84BE247D8D7E247DC57FE
:102BD00029471D8FE24798CFE247D85797E7010072
:102BE000938707A29C4363F9E700E247D85797E72A
:102BF00001009387E7A098C3E247D857BA878A07AE
:102C0000BA978A0717E701001307878B3E97E247B9
:102C10009107BE853A85EFD03F9985473ECEF24772
:102C20003E85B250456182807370043097E70100A1
:102C30009387479D9C4391CF97D701009387077B4C
:102C40009C43F8430507F8C397D701009387077A99
:102C50009C430100828097E701009387A79A9C43D9
:102C60008DCB97D70100938767789C43FC4395C32E
:102C700097D70100938787779C43F8437D17F8C364
:102C800097D70100938787769C43FC4399E3736051
:102C9000043001008280411197D7010093870775A6
:102CA0009C439C4F3EC697D70100938727749C4353
:102CB000D85797D70100938767739C43A9463387FA
:102CC000E64098CFB2473E854101828097D7010008
:102CD0009387C7719C4389CB97D70100938707716E
:102CE0009C43F84B0507F8CB97D7010093870770F3
:102CF0009C433E858280797106D62AC62EC42D3724
:102D000097D701009387876E9C43BC4FADE397D75D
:102D100001009387A76D9C430547F8CFA247A1CB3D
:102D200097D701009387876C9C4391073E85EFD02E
:102D30005F922247FD576310F70297D701009387F0
:102D4000E76A9C439107BE8517E501001305858955
:102D5000EFD09F8519A897E701009387278A9C43A6
:102D60002247BA973ECE7245353CEFD02FEAE53583
:102D7000653D97D70100938767679C43BC4F3ECC66
:102D8000E2479DC3B24789CB97D701009387076677
:102D90009C4323AC070409A897D7010093870765D4
:102DA0009C43B84F7D17B8CF97D70100938707642E
:102DB0009C4323AE07044535E2473E85B25045614A
:102DC0008280797106D62AC62EC432C236C0A93D89
:102DD00097D70100938787619C43F84F8947630D1C
:102DE000F70697D70100938767609C43B44F32473B
:102DF0001347F7FF758FB8CF97D701009387075F09
:102E00009C430547F8CF8247A1CB97D70100938712
:102E1000E75D9C4391073E85EFD0BF830247FD5796
:102E20006310F70297D701009387475C9C43910793
:102E3000BE8517D501001305E57AEFD0EFF619A886
:102E400097D701009387877B9C430247BA973ECC74
:102E50006245893AEFD08FDBFD3BF933924789CB4E
:102E600097D70100938787589C43B84F924798C3E0
:102E700097D70100938787579C43F84F8547631482
:102E8000F70002CE31A897D70100938727569C43BD
:102E9000B44F22471347F7FF758FB8CF85473ECE13
:102EA00097D70100938787549C4323AE070465336B
:102EB000F2473E85B25045618280797106D62AC6B6
:102EC0002EC432C236C085473ECEB24781E773700A
:102ED000043001A0B2473ECC813B824789C7E2471C
:102EE000B84F824798C3E247FC4F3ECAE2470947C2
:102EF000F8CF1247914763EEE704924713972700F4
:102F000097D7010093878710BA97984397D7010006
:102F10009387C70FBA978287E247B84FA2475D8F62
:102F2000E247B8CF3DA0E247BC4F13871700E24706
:102F3000B8CF05A0E2472247B8CF21A8524789471A
:102F40006306F700E2472247B8CF21A002CE11A0C6
:102F5000010052478547631AF706E24791073E850D
:102F6000EFD02FEFE247D85797D7010093874769F3
:102F70009C4363F9E700E247D85797D7010093874E
:102F8000276898C3E247D857BA878A07BA978A074B
:102F900017D701001307C7523E97E2479107BE8536
:102FA0003A85EFD06FE0E2479C5781C773700430D9
:102FB00001A0E247D85797D70100938727439C4346
:102FC000DC5763F4E700EFD06FC47131F2473E8500
:102FD000B25045618280397106DE2ACE2ECC32CACB
:102FE00036C83AC685473ED6F24781E7737004304B
:102FF00001A0F2473ED4EFD04FCFAA873ED2C247BE
:1030000089C7A257B84FC24798C3A257FC4F3ED0BA
:10301000A2570947F8CF5247914763EEE704D247DA
:103020001397270097D70100938787FFBA97984394
:1030300097D701009387C7FEBA978287A257B84FE8
:10304000E2475D8FA257B8CF3DA0A257BC4F138770
:103050001700A257B8CF05A0A2576247B8CF21A842
:10306000025789476306F700A2576247B8CF21A0ED
:1030700002D611A0010002578547631DF708A25729
:103080009C5781C77370043001A097D701009387C4
:10309000E7589C43A1EBA25791073E85EFD06FDB29
:1030A000A257D85797D70100938787559C4363F958
:1030B000E700A257D85797D701009387675498C362
:1030C000A257D857BA878A07BA978A0717D7010035
:1030D0001307073F3E97A2579107BE853A85EFD069
:1030E000AFCC11A8A257E107BE8517D50100130583
:1030F000A54CEFD06FCBA257D85797D70100938735
:10310000E72E9C43DC5763F7E700B24781C7B2471D
:10311000054798C392573E85EFD02FBCB2573E85E6
:10312000F25021618280797106D62AC62EC4B24738
:1031300081E77370043001A0B2473ECEEFD0EFBA02
:10314000AA873ECCF247FC4F3ECAF2470947F8CF68
:10315000F247BC4F13871700F247B8CF5247854755
:10316000631DF708F2479C5781C77370043001A0B4
:1031700097D701009387874A9C43A1EBF2479107B9
:103180003E85EFD00FCDF247D85797D701009387F0
:1031900027479C4363F9E700F247D85797D70100C8
:1031A0009387074698C3F247D857BA878A07BA97D2
:1031B0008A0717D701001307A7303E97F2479107F8
:1031C000BE853A85EFD04FBE11A8F247E107BE8514
:1031D00017D501001305453EEFD00FBDF247D85774
:1031E00097D70100938787209C43DC5763F7E7005C
:1031F000A24781C7A247054798C3E2473E85EFD063
:10320000CFAD0100B25045618280797106D62AC6E1
:10321000B2473ECCE24799E797D701009387071D55
:103220009C4311A0E2473ECC0134E247F84F894766
:103230006318F700E24723AE070485473ECE11A08E
:1032400002CE113CF2473E85B250456182800111A9
:1032500006CE02C61D2B97D701009387673F9C437C
:103260009DC38148014881470947814613060040B4
:1032700097D50100938505DC170500001305051B94
:10328000EFE0AF852AC6B24781E77370043001A032
:10329000B2473E85F24005618280397106DE2ACE52
:1032A0002ECC32CA36C83AC6E24799E302D62DA8D8
:1032B0001305C002EF00302A2AD6B25795C7F12174
:1032C000B257724798C3B257624798CFB257524726
:1032D000D8CFB257424798D3B2573247D8D3B25714
:1032E00091073E85EFD04FABE24781E77370043022
:1032F00001A0B2573E85F25021618280397106DE0D
:103300002ACE2ECC32CA36C83AC602D6F24781E758
:103310007370043001A097D70100938767339C43F3
:10332000B5CBE2473ED0D2473ED2F2473ED46247C9
:10333000954763C4E704EFF0AFF22A87894763102B
:10334000F70297D701009387A7309C431810814656
:103350003246BA853E85EFD0AFE02AD625A897D76A
:1033600001009387E72E9C43181081460146BA85D9
:103370003E85EFD0EFDE2AD631A897D7010093879C
:10338000272D9C43181081464246BA853E85EFD0D2
:103390000FF32AD6B2573E85F25021618280011187
:1033A0002AC6B2473ECEB24781E77370043001A00F
:1033B000F2479C433E8505618280797106D62AC614
:1033C0002EC497D70100938727289C43DC47DC470E
:1033D0003ECEF24791073E85EFD0AFA7F247D84FD8
:1033E0008547631BF702F247984FB247BA97B24638
:1033F0002246BE857245B9222A878547631EF7009B
:1034000001478146324681457245CD3D2ACCE2478F
:1034100081E77370043001A0F247DC537245829754
:103420000100B25045618280797106D62AC63C08F7
:103430003E8541282ACEE247BE8572451920692281
:10344000FDB7797106D62AC62EC4EFE06FF93C08A5
:103450003E8545282ACEE247B9EFA24799EB32478D
:10346000F24763E8E700EFE06FF9F2453245B13724
:10347000A9A0A24781CF97D701009387271D9C431E
:103480009C4393B7170093F7F70F3EC497D70100FB
:103490009387071C94433247F247B307F74022460D
:1034A000BE853685EFD0FFDDEFE04FF5AA8791E7C7
:1034B000EFC0DFF519A0EFE06FF40100B2504561F5
:1034C000828001112AC697D701009387E7179C4392
:1034D0009C4393B7170093F7F70F3E87B24798C303
:1034E000B2479C4391EB97D701009387E7159C4324
:1034F000DC479C433ECE11A002CEF2473E850561DB
:103500008280797106D62AC6EFE01F842ACE97D72B
:103510000100938727149C4372476377F700692A59
:10352000B247054798C321A0B24723A0070097D709
:10353000010093872712724798C3F2473E85B25025
:1035400045618280797106D62AC62EC432C236C041
:1035500002CEB2472247D8C3B247324798CB224760
:10356000924763E8E702124782471D8FB2479C4F9C
:103570006365F70085473ECE99A097D701009387F2
:10358000E70C9843B2479107BE853A85EFD0CF85C7
:103590003DA0124782476379F7002247824763655F
:1035A000F70085473ECE21A897D701009387C7092A
:1035B0009843B2479107BE853A85EFD0EF82F24734
:1035C0003E85B25045618280797106D6D9A0A24766
:1035D00063C0070CC2473ECEF247DC4B91C7F247AF
:1035E00091073E85EFD0EF865C003E85193F2ACCDF
:1035F000A2472547636FF7081397270097D7010065
:103600009387C7A3BA97984397D70100938707A3D7
:10361000BA9782873247F2479C4FBA973247BA86A9
:103620006246BE857245393F2A8785476313F70690
:10363000F247DC5372458297F247D84F8547631AA9
:10364000F7043247F2479C4FBA97014781463E86BE
:103650008145724565312ACAD24785EF73700430BF
:1036600001A03247F24798CFF2479C4F81E7737031
:10367000043001A0F247984FE247BA97E24662460B
:10368000BE857245C13531A07245EF00C07F11A0E3
:10369000010097D701009387A7FB9C433800814620
:1036A0000146BA853E85EFD06FD8AA87E39107F22D
:1036B0000100B25045618280797106D671A097D71A
:1036C0000100938767F89C43DC479C433ECC97D727
:1036D0000100938767F79C43DC47DC473ECAD2472B
:1036E00091073E85EFC0FFF6D247DC5352458297E3
:1036F000D247D84F85476319F704D2479C4F62479A
:10370000BA973EC84247E24763F4E702D2474247CE
:10371000D8C3D247524798CB97D701009387C7F2B7
:103720009843D2479107BE853A85EFC0FFEB29A8A1
:1037300001478146624681455245C9362AC6B2478D
:1037400081E77370043001A097D701009387C7EF1A
:103750009C439C43ADF797D701009387E7EE9C43CA
:103760003ECE97D70100938767EE984397D7010025
:10377000938787ED98C397D70100938727ED72470A
:1037800098C30100B25045618280411106C6EFF036
:10379000AFC997D701009387A7EB9C43C9E717D51B
:1037A00001001305E5E7EFC0FFDB17D501001305A6
:1037B00065E8EFC03FDB97D701009387E7E817D7AD
:1037C00001001307E7E598C397D70100938707E83F
:1037D00017D70100130707E698C30146B145114505
:1037E000EFC07FF72A8797D70100938767E698C3D2
:1037F00097D701009387C7E59C4381E77370043036
:1038000001A097D701009387A7E49C4389CF97D75E
:1038100001009387E7E39C4397D501009385858456
:103820003E85EFD05F9CEFF00FC30100B240410135
:103830008280797106D62AC6B2473ECEB24781E76A
:103840007370043001A0EFF02FBEF247DC4BB337AA
:10385000F00093F7F70F3ECCEFF0EFBFE2473E8565
:10386000B25045618280797106D62AC6B2473ECEF3
:10387000B24781E77370043001A0EFF0EFBAF2476E
:103880009C533ECCEFF02FBDE2473E85B2504561E0
:103890008280797106D62AC62EC4B2473ECEB24780
:1038A00081E77370043001A0EFF00FB8F2472247B0
:1038B00098D3EFF04FBA0100B250456182800111F8
:1038C00006CE714549292AC6B24789CBB24723A003
:1038D0000700B24791073E85EFC0DFC8B2473E857B
:1038E000F24005618280397106DE2AC62EC432C2DA
:1038F00036C0B2473ED402D21247B70700FFF98F55
:1039000081C77370043001A0924781E7737004305F
:1039100001A0EFF0EF94AA8799E3824799E38547E6
:1039200011A0814781E77370043001A0EFE04FAB35
:10393000A2579C433ED0A245324585240257A24758
:103940005D8F9247F98F12476310F7020257A24723
:10395000D98F3ED6A2579843924793C7F7FF7D8FE2
:10396000A25798C302C025A0824799CFA257938639
:1039700047001247B7070005D98F0246BE85368536
:10398000EFE03F8902D621A0A2579C433ED6EFE04C
:10399000EFA62ACE8247B1CBF24799E3EFC01FA72B
:1039A000EFF06FAF2AD63257B7070002F98F85EBD9
:1039B000EFF08FA7A2579C433ED632579247F98F1C
:1039C0001247631AF700A2579843924793C7F7FF2D
:1039D0007D8FA25798C3EFF00FA885473ED232578C
:1039E000B7070001FD17F98F3ED6B2573E85F2505A
:1039F000216182805D7186C62ACE2ECC32CA36C83D
:103A00003AC6F2473EDA02DC02D8F24781E7737029
:103A1000043001A06247B70700FFF98F81C77370B8
:103A2000043001A0E24781E77370043001A0EFF099
:103A30002F83AA8799E3B24799E3854711A081476D
:103A400081E77370043001A0EFE08F99D2579C4357
:103A50003ED64246E245325575242AD4A25799CF24
:103A6000B2573EDE02C6D247A9CBD2579843E247AF
:103A700093C7F7FF7D8FD25798C381A0B24781E7E4
:103A8000B2573EDE1DA8D24791C76257B707000163
:103A9000D98F3EDCC24791C76257B7070004D98F60
:103AA0003EDCD257938647006247E257D98F3246B1
:103AB000BE853685EFE0EFF502DEEFE02F942AD2E7
:103AC000B247B9CB925799E3EFC05F94EFF0AF9C48
:103AD0002ADE7257B7070002F98F8DEBEFF0CF9413
:103AE000D2579C433EDE4246E2457255212CAA87BE
:103AF00099CBD24789CBD2579843E24793C7F7FF78
:103B00007D8FD25798C3EFF00F9502D87257B70741
:103B10000001FD17F98F3EDEF2573E85B640616128
:103B20008280797106D62AC62EC4B2473ECEB247ED
:103B300081E77370043001A02247B70700FFF98FB7
:103B400081C77370043001A0EFF00F8EF2479C43E1
:103B50003ECCF2479843A24793C7F7FF7D8FF247C9
:103B600098C3EFF04F8FE2473E85B25045618280A7
:103B7000797106D62AC6B2473ECEEFC01F97AA87F4
:103B80003ECCF2479C433ECAE2473E85EFC0FF94DD
:103B9000D2473E85B250456182805D7186C62AC695
:103BA0002EC402DCB2473ED802DAB24781E7737016
:103BB000043001A02247B70700FFF98F81C7737057
:103BC000043001A0C25791073ED6B257A1073ED498
:103BD000EFE00F81B257DC473EDEC2579843A24761
:103BE0005D8FC25798C3BDA8F257DC433ED2F2574F
:103BF0009C433ED002DA0257B70700FFF98F3ECE52
:103C00000257B7070001FD17F98F3ED07247B7077B
:103C10000004F98F89EBC25798438257F98F89CFF7
:103C200085473EDA11A8C25798438257F98F025749
:103C30006314F70085473EDAD2579DC37247B70732
:103C40000001F98F89C762578257D98F3EDCC2576E
:103C50009843B7070002D98FBE857255EFE00FF980
:103C600092573EDE7257A257E310F7F8C2579843B7
:103C7000E25793C7F7FF7D8FC25798C3EFD01FF865
:103C8000C2579C433E85B64061618280797106D6F9
:103C90002AC6B2473ECEF24791073ECCEFD05FF442
:103CA0000DA0E247D847E247A1076315F7007370FC
:103CB000043001A0E247DC47B70500023E85EFE093
:103CC000EFF2E2479C43F1FF7245752AEFD01FF3F4
:103CD0000100B25045618280011106CE2AC62EC471
:103CE000A24532455D3D0100F2400561828001112F
:103CF00006CE2AC62EC4A245324525350100F24023
:103D00000561828001112AC62EC432C202CE9247BA
:103D100081EB3247A247F98F81CF85473ECE09A874
:103D20003247A247F98F22476314F70085473ECEFA
:103D3000F2473E850561828001112AC6B2473ECC1A
:103D4000B24799E302CE21A0E2479C4F3ECEF24714
:103D50003E8505618280397106DE2AC602D2EFD027
:103D60003FE897670300938727909C4381EB552298
:103D7000976703009387478F054798C3B24789CF5A
:103D8000A1473E87B247BA973EC6B2478D8B89C7D7
:103D9000B247F19B91073EC6B247F9CB3247E56780
:103DA000ED1763E7E70C976703009387E78A3ED434
:103DB000976703009387478A9C433ED631A0B2574A
:103DC0003ED4B2579C433ED6B257DC43324763F5EC
:103DD000E700B2579C43E5F7325797670300938794
:103DE00027886307F708A2579C432147BA973ED21A
:103DF000B2579843A25798C3B257D843B247B307B4
:103E0000F740214706076378F7043257B247BA975D
:103E10003ECEB257D843B2471D8FF247D8C3B257F0
:103E20003247D8C3F247DC433ECC97670300938701
:103E3000A7823ED021A082579C433ED082579C430C
:103E4000DC436247E3E9E7FE82579843F24798C3B1
:103E50008257724798C397C701009387675A984360
:103E6000B257DC431D8F97C701009387675998C3EA
:103E7000EFD0DFD8925799E3EF00D03192573E85CB
:103E8000F25021618280797106D62AC6B2473ECCB3
:103E9000B247BDC3A147B307F0406247BA973ECCD3
:103EA000E2473ECAEFD0DFD3D247DC433EC8975744
:103EB00003009387677A3ECE21A0F2479C433ECE13
:103EC000F2479C43DC434247E3E9E7FEF24798436D
:103ED000D24798C3F247524798C3D247D84397C7AF
:103EE00001009387E7519C433E9797C70100938752
:103EF000275198C3EFD09FD00100B2504561828016
:103F000097C701009387C74F9C433E85828001007D
:103F10008280411197C7010093874774F19B3EC689
:103F20009757030093874773324798C39757030007
:103F30009387877223A207009757030093874772DE
:103F400065677117D8C3975703009387677123A0DC
:103F50000700B2473EC4A24765677117D8C3A2479E
:103F6000175703001307C76F98C3010041018280F0
:103F700001112AC62EC432C2A2473ECEB2473ECC61
:103F80003247A247D98F8D8BA1E319A8F2479843F6
:103F9000E24798C3E24791073ECCF24791073ECEF5
:103FA0009247F5173247BA976247E361F7FE29A8AF
:103FB0007247930717003ECEE2479386170036CC30
:103FC000034707002380E70032479247BA976247CA
:103FD000E360F7FEB2473E850561828001112AC683
:103FE0002EC432C232479247D98F8D8B9DEFA247A4
:103FF00093F7F70F3ECAD247A2075247D98F3ECA5E
:10400000D247C2075247D98F3ECAB2473ECE39A0E7
:10401000F247138747003ACE524798C33247924738
:10402000BA977247E366F7FE1DA0B2473ECC11A8CF
:10403000E247138717003ACC22471377F70F238004
:10404000E70032479247BA976247E363F7FEB24709
:104050003E850561828001112AC6B2473ECE21A06D
:10406000F24785073ECEF24783C70700F5FB72474C
:10407000B247B307F7403E850561828001112AC629
:104080002EC4B247138717003AC683C70700A30F91
:10409000F100A247138717003AC483C70700230F14
:1040A000F1008347F10199C70347F1018347E1011B
:1040B000E309F7FC0347F1018347E101B307F74048
:1040C0003E850561828001112AC62EC4B2473ECECC
:1040D00001002247930717003EC4F247938617005A
:1040E00036CE034707002380E70083C70700F5F3B8
:1040F000B2473E850561828001112AC602CE02CCFC
:1041000021A0B24785073EC6B24703C70700930701
:104110000002E308F7FEB24703C707009307D00287
:104120006309F700B24703C707009307B0026311A2
:10413000F704B24783C70700938737FD93B717008B
:1041400093F7F70F3ECCB24785073EC615A07247DE
:10415000BA878A07BA9786073ECEB24713871700F9
:104160003AC683C70700938707FD7247BA973ECECA
:10417000B24783C70700E1FFE24789C7F247B307A9
:10418000F04011A0F2473E850561828001112AC6E8
:10419000975703009387074F9C4393861700175741
:1041A00003001307274E14C332471377F70F9756B0
:1041B000030093862651B6972380E7003247A9472C
:1041C000630BF700975703009387C74B98439307F8
:1041D00000046315F704975703009387A74E3ECE5C
:1041E00005A8F247138717003ACE03C70700B707A1
:1041F00010F0938707F098C3975703009387874879
:104200009C431387F7FF975703009387A74798C3EB
:1042100097570300938707479C43E1F781473E8503
:10422000056182804D7123261114232481142322D9
:10423000911423202115232E3113232C4113232ADB
:1042400051132ACE2ECC32C836CA3AC63EC442C218
:1042500023260112B2473E8A814AC24752485286FB
:10426000D6863E85C285EF10E020AA872E883E863E
:10427000C2868327C112138717002326E1123287D3
:104280008A07141AB69723AEE7EEB2473E848144FC
:10429000D247268763E8E702D24726876396E7007E
:1042A000C247228763E0E702B2473E8981494A86D6
:1042B000CE864245D245EF00303EAA872E883EC8C2
:1042C00042CA49BF010029A0F247E2451245829740
:1042D000A2471387F7FF3AC40327C112E346F7FE4C
:1042E00025A88327C1128A07181ABA9703A7C7EF10
:1042F0008327C1128A07141AB69783A6C7EFA5476A
:1043000063F5D7009307700519A093070003BA97C8
:104310007247E2453E8502978327C1121387F7FF54
:104320002326E112E34FF0FA01008320C114032495
:10433000811483244114032901148329C113032AFE
:104340008113832A41137161828041112AC62EC4D0
:10435000A2460547635ED700B2479C439D07E19B99
:1043600093868700324714C303A847009C4335A0B7
:10437000224719CB3247184313064700B24690C272
:104380001843BA87014811A832471843130647005B
:10439000B24690C21843BA8701483E85C2854101A2
:1043A000828041112AC62EC4A2460547635ED7000B
:1043B000B2479C439D07E19B93868700324714C315
:1043C00003A847009C4305A8224701CF3247184362
:1043D00013064700B24690C21843BA877D873A88D1
:1043E00019A83247184313064700B24690C2184333
:1043F000BA877D873A883E85C285410182803971BE
:1044000006DE22DC26DA2AC62EC432C236C011A845
:1044100063070424924785073EC2B247A24522851E
:104420008297924783C707003E8493075002E311A7
:10443000F4FE924785073EC292473EC893070002AA
:10444000A30BF100FD573ECEFD573ECC02D0924764
:10445000138717003AC283C707003E849307D4FD31
:10446000130750056364F71E1397270097C70100D1
:10447000938747C0BA97984397C70100938787BF30
:10448000BA9782879307D002A30BF100C9B79307AD
:104490000003A30BF10065BF02CC6247BA878A070D
:1044A000BA978607A297938707FD3ECC924783C7AA
:1044B00007003E849307F00263D6870293079003B8
:1044C00063C28702924785073EC2C1BF82471387F6
:1044D00047003AC09C433ECC39A0F247E3D907F6E7
:1044E00002CEB5B70100F247E3D307F6E2473ECE6E
:1044F000FD573ECCA9BF825785073ED089BF824772
:10450000138747003AC09C433247A2453E85029735
:10451000B1A28247138747003AC0844389E497C415
:1045200001009384A4B4F2476357F0040347710178
:104530009307D0026301F704E247BE852685EF00AA
:1045400070132A87F247998F3ECE11A883477101D5
:104550003247A2453E850297F247FD173ECEF2470D
:10456000E346F0FE09A8B247A2452285829785045A
:10457000F247FD173ECE83C704003E841DC0E247CC
:10458000E3C307FEE247FD173ECCE247E3DD07FC4D
:1045900009A8B247A245130500028297F247FD170A
:1045A0003ECEF247E347F0FE55A88A8782553E8506
:1045B000CD3BAA872E883ED442D6A2573258C28716
:1045C00063D90702B247A2451305D0028297A255CC
:1045D000325681470148B386B740368533B5A700C8
:1045E0003307C840B307A7403E87B6873A883ED412
:1045F00042D6A9473ED21DA8A9473ED215A0A14741
:104600003ED239A885473ED0B247A24513050003E4
:104610008297B247A245130580078297C1473ED2D1
:104620008A8782553E8515332AD42ED61257834762
:1046300071013E88F2472256B256A2453245DD3618
:1046400031A8B247A2452285829709A8B247A24560
:10465000130550028297C2473EC20100D9B3010040
:10466000F2506254D2542161828041112AC6B707A8
:1046700010F0938707F2324798C301A05D7106D608
:104680002AC62EDA32DC36DEBAC0BEC2C2C4C6C604
:104690009C0891173ECEF247BE86324681451705EB
:1046A00000001305E5AEA13B81473E85B250616134
:1046B000828001112AC62EC41EC2A2473ECEF247F6
:1046C0009C4332471377F70F2380E700F2479C4360
:1046D00013871700F24798C30100056182801D719E
:1046E00006DE2AC62EC4B2C4B6C6BAC8BECAC2CC7A
:1046F000C6CE9C103ED25C084C081706000013067C
:1047000086FB7D779346F7FF0565130505803388A3
:10471000A5003378E8001368783B23A007013295A1
:10472000698F13677733D8C333F7D50093154701E3
:1047300037870300130737394D8F98C73377D60073
:10474000931647013707030013077706558FD8C71D
:104750000F100000B2473ED69C10A1173ED422573E
:104760005C083E857C00BA862246BE854939B24740
:1047700023800700B2473E87B257B307F7403E8514
:10478000F250256182804111370510F0130545F480
:1047900008412AC6370510F0130505F408412AC45C
:1047A000370510F0130545F40841B248E39EA8FC14
:1047B00032452A8381431317030081462245AA8587
:1047C0000146B3E7B6003368C700370710F013059A
:1047D00087F48565938505FA0146B386B700B688E8
:1047E000B3B8F8003307C800B387E8003E87B68740
:1047F0003A881CC123220501010041018280411138
:1048000006C651379307000873A047300100B24035
:1048100041018280011106CE2AC617C50100130589
:10482000E59AEFF0BFE50100F240056182800111D9
:1048300006CE2AC617C501001305C599EFF01FE47F
:104840000100F24005618280797106D62AC602CE47
:1048500029A00100F24785073ECE724785679387FE
:104860007738E3D8E7FE17C5010013052597EFF069
:10487000FFE0F1BF411106C60D2A0100B24041011F
:104880008280011106CE02C6312B2A878547630C30
:10489000F70017C501001305E594EFF03FDEB247BE
:1048A00093E727003EC6B2473E85F240056182800D
:1048B000011106CE02C67D3F1707000013076704EB
:1048C000814605469305400617C50100130545932B
:1048D000EFE0BF9C2AC6B24799CBEFD0EFC6AA87BC
:1048E000014781463E8685453245EFE03FA102C43F
:1048F000EFD02FA581473E85F24005618280797116
:1049000006D62AC697C70100938787AE9C431387B4
:10491000470697C701009387A7AD98C397C70100C3
:10492000938747AD9C431387470697C7010093873A
:1049300067AC98C397C70100938787AB98439307E9
:10494000F07C63D3E70497C70100938767AA9C4371
:104950001387078397C70100938787A998C31537E3
:104960002ACEF24799EB97C701009387A7A89843EF
:1049700085679387F77663DBE700F2473E85EFF0C4
:10498000DFCEEFD0EFA321A0010011A00100B250B3
:10499000456182807370043001A001008280411162
:1049A0002AC62EC47370043001A0411106C61145F9
:1049B000EFB03FE32A87975703009387A7D498C3A4
:1049C00097570300938707D49C4397C501009385AD
:1049D000E5833E85EFC03F8197570300938787D2D9
:1049E0009C43B5CB8148014897570300938747D331
:1049F000094781461306004097C50100938505824B
:104A0000170500001305E505EFC03F8D81480148FB
:104A100097570300938707D1054781461306004047
:104A200097C50100938505801705000013056513E0
:104A3000EFC0BF8A8148014881470147814613067C
:104A4000004097B501009385657E170500001305AA
:104A5000451EEFC09F880100B240410182807971FC
:104A600006D62AC6975703009387C7C99C433E853D
:104A7000EFB01FDF2A8785476318F70097570300B9
:104A8000938787C8054798C302CE15A89757030098
:104A9000938747C79C43A1453E85EFB0BFE12A8776
:104AA00085476308F700975703009387E7C50547D5
:104AB00098C35145EFC09FB5F24785073ECE724778
:104AC000A547E3F5E7FC02CE0DA85145EFC01FB4A2
:104AD00097570300938707C39C433E85EFB05FD889
:104AE0002A8785476308F700975703009387C7C154
:104AF000054798C3F24785073ECE7247A547E3F6C0
:104B0000E7FC975703009387E7BF9C433E85EFB0D0
:104B10003FD52A8785476318F70097570300938787
:104B2000A7BE054798C3975703009387A7BE9C432A
:104B300013871700975703009387C7BD98C39757EC
:104B400003009387A7BC054798C30145EFC0DFD694
:104B500097570300938787BB23A0070021B7011154
:104B600006CE2AC6975703009387C7B99C43F955C9
:104B70003E85EFB03FD42A8785476313F7069757E2
:104B800003009387A7B8984385476309F7009757B1
:104B90000300938767B7054798C389A89757030011
:104BA000938747B69C433E85EFB09FCB2A878547C6
:104BB0006308F70097570300938707B5054798C325
:104BC000975703009387C7B4054798C30145EFC0C3
:104BD000BFCE975703009387A7B323A0070039A040
:104BE00097570300938747B2054798C39757030029
:104BF000938787B29C4313871700975703009387C7
:104C000067B19C436308F700975703009387C7AFCA
:104C1000054798C397570300938707B09C431387B2
:104C2000170097570300938727AF98C325BF01113B
:104C300006CE2AC6975703009387C7AC9C4381458D
:104C40003E85EFB03FC72A878547E315F7FE9757A4
:104C500003009387E7AC9C433E85EFC0FFA02A8703
:104C60008D476305F7007370043001A09757030068
:104C7000938747AB9C433E85EFC01F9F2A878D4794
:104C80006305F7007370043001A097570300938702
:104C900027A898438547631AF7009757030093871F
:104CA000E7A6984385476309F70097570300938762
:104CB000A7A5054798C3F5A097570300938707A6B4
:104CC0009C431387170097570300938727A598C322
:104CD00097570300938707A59C433E85EFC0FFCFFE
:104CE000975703009387C7A39C433E85EFC0FFCE31
:104CF000975703009387C7A198438547630AF70036
:104D000097570300938787A0984385476318F70058
:104D1000975703009387479F054798C30145EFC006
:104D20009F9E2A8789476305F7007370043001A0AE
:104D3000975703009387C79E9C433E85EFC0DF9241
:104D40002A8789476305F7007370043001A09757DD
:104D500003009387279D9C433E85EFC0FF902A87E1
:104D600089476305F7007370043001A0975703006B
:104D7000938747999C433E85EFB09FAE2A8785472E
:104D80006308F7009757030093870798054798C370
:104D90000145EFC05F97AA87E38E07E87370043080
:104DA00001A049BD4111975703009387E7979843A6
:104DB00097570300938707969C436319F70097570B
:104DC000030093876794054798C319A89757030072
:104DD000938747949843975703009387E79498C322
:104DE00097570300938787949843975703009387B7
:104DF000A7929C436319F700975703009387C790C6
:104E0000054798C319A8975703009387E7909843DD
:104E1000975703009387879198C397570300938709
:104E200027919843975703009387478F9C436319B3
:104E3000F700975703009387278D054798C319A854
:104E4000975703009387878D98439757030093875D
:104E5000278E98C3975703009387078B98438547FE
:104E60006314F70002C619A085473EC6B2473E85C7
:104E700041018280B305B500930705006386B70042
:104E800003C70700631607003385A740678000004B
:104E9000938717006FF09FFE130101FD23229102FB
:104EA000232A5101232611022324810223202103D6
:104EB000232E3101232C4101232861012326710176
:104EC00023248101232291012320A101930A0500BB
:104ED00093840500639E06381304060093090500B9
:104EE00017B901001309093563F8C512B7070100A6
:104EF000138B05006378F6101307F00F3337C700E4
:104F000013173700B357E6003309F9008346090049
:104F10003387E60093060002B386E640638C060002
:104F2000B394D40033D7EA003314D600336B970020
:104F3000B399DA00935A040193850A0013050B0014
:104F4000EF00902A1309050093850A00931B0401C2
:104F500013050B00EF00D02493DB0B019304050035
:104F60009305050013850B00EF00D02013190901EC
:104F700093D70901B367F900138A040063FEA70001
:104F8000B3878700138AF4FF63E8870063F6A700FE
:104F9000138AE4FFB3878700B384A74093850A0090
:104FA00013850400EF0050241309050093850A00BF
:104FB00013850400EF00D01E9399090193040500A6
:104FC000930505001319090113850B0093D90901F5
:104FD000EF00501AB36939011386040063FCA9007D
:104FE000B30934011386F4FF63E6890063F4A90072
:104FF0001386E4FF13140A013364C400130A00008B
:105000006F000013B707000113070001E36CF6EE11
:10501000130780016FF01FEF138A0600631A060062
:105020009305000013051000EF009017130405000E
:10503000B7070100637EF4129307F00F63F4870053
:10504000130A8000B35744013309F90003470900EC
:105050009306000233074701B386E64063940612C5
:10506000B3848440130A1000135B040193050B0002
:1050700013850400EF0050171309050093050B007A
:1050800013850400931B0401EF00901193DB0B01C7
:10509000930405009305050013850B00EF00900DA8
:1050A0001319090193D70901B367F900938A040022
:1050B00063FEA700B3878700938AF4FF63E8870045
:1050C00063F6A700938AE4FFB3878700B384A74001
:1050D00093050B0013850400EF0010111309050060
:1050E00093050B0013850400EF00900B93990901C1
:1050F00093040500930505001319090113850B009E
:1051000093D90901EF001007B36939011386040030
:1051100063FCA900B30934011386F4FF63E6890038
:1051200063F4A9001386E4FF13940A013364C400F6
:105130001305040093050A008320C10203248102A1
:1051400083244102032901028329C101032A810129
:10515000832A4101032B0101832BC100032C810011
:10516000832C4100032D010013010103678000001F
:10517000B7070001130A0001E366F4EC130A80018B
:105180006FF05FEC3314D40033DAE400B399DA0043
:1051900033D7EA00935A0401B394D40093850A00EC
:1051A00013050A00336B9700EF0010041309050084
:1051B00093850A0013050A00931B0401EF00407E4B
:1051C00093DB0B01930405009305050013850B0089
:1051D000EF00407A1319090113570B013367E900F7
:1051E000138A0400637EA70033078700138AF4FF45
:1051F000636887006376A700138AE4FF330787009C
:10520000B304A74093850A0013850400EF00C07D16
:105210001309050093850A0013850400EF00407808
:10522000930405009305050013850B00EF008074BF
:1052300013170B011357070113190901B367E9008D
:105240001387040063FEA700B38787001387F4FF6A
:1052500063E8870063F6A7001387E4FFB38787003E
:10526000131A0A01B384A740336AEA006FF0DFDF44
:1052700063ECD51EB707010063F4F6041307F00FC3
:10528000B335D7009395350033D7B60097B70100F3
:10529000938747FAB387E70003C70700130A0002A2
:1052A0003307B700330AEA4063160A0213041000FA
:1052B000E3E096E833B6CA00134416006FF05FE7E8
:1052C000B707000193050001E3E0F6FC93058001B8
:1052D0006FF09FFBB35CE600B3964601B3ECDC00D5
:1052E00033D4E40093DB0C01B397440133D7EA00D5
:1052F00093850B0013050400336BF700B3194601C7
:10530000EF00806E1309050093850B001305040060
:10531000139C0C01EF00C068135C0C0193040500A2
:105320009305050013050C00EF00C0641319090173
:1053300013570B013367E90013840400637EA70051
:10534000330797011384F4FF636897016376A7001E
:105350001384E4FF33079701B304A74093850B0040
:1053600013850400EF0040681309050093850B00C6
:1053700013850400EF00C062930405009305050047
:1053800013050C00EF00005F93170B0113190901BF
:1053900093D70701B367F9001386040063FEA700E3
:1053A000B38797011386F4FF63E8970163F6A700BC
:1053B0001386E4FFB387970113140401B70B0100B0
:1053C0003364C4001389FBFF337D240133F92901C1
:1053D000B384A7409305090013050D00EF00805921
:1053E000935C040193050900130B050013850C0061
:1053F000EF00405893D90901130C0500938509006B
:1054000013850C00EF000057130905009385090070
:1054100013050D00EF0000563305850193570B016E
:105420003385A7006374850133097901935705011A
:10543000B387270163E6F402E392F4BCB7070100E7
:105440009387F7FF3375F50013150501337BFB00D8
:1054500033964A0133056501130A0000E37AA6CCAE
:105460001304F4FF6FF09FB9130A00001304000047
:105470006FF01FCC130101FB23248104232291042C
:10548000232E3103232291032326110423202105F7
:10549000232C4103232A510323286103232671036C
:1054A000232481032320A103232EB101930C0500A3
:1054B000938905001304050093840500639E062666
:1054C00013090600138A060097BA0100938A8AD648
:1054D00063F4C514B70701006376F6129307F00F63
:1054E00063F4C700130A8000B3574601B38AFA0079
:1054F00003C70A001305000233074701330AE540DA
:10550000630C0A00B395490133D7EC003319460107
:10551000B364B70033944C01935A090193850A0090
:1055200013850400EF00404C9309050093850A00A1
:10553000131B090113850400EF008046135B0B0168
:105540009305050013050B00EF00C0429399090174
:1055500093570401B3E7F90063FAA700B387270163
:1055600063E6270163F4A700B3872701B384A7404C
:1055700093850A0013850400EF0000479309050096
:1055800093850A0013850400EF0080411314040181
:10559000930505009399090113050B0013540401A9
:1055A000EF00403D33E48900637AA4003304240112
:1055B000636624016374A400330424013304A4400B
:1055C00033554401930500008320C1040324810462
:1055D00083244104032901048329C103032A81038D
:1055E000832A4103032B0103832BC102032C810275
:1055F000832C4102032D0102832DC10113010105FA
:1056000067800000B7070001130A0001E36EF6ECA3
:10561000130A80016FF05FED631A06009305000026
:1056200013051000EF00C03713090500B70701008C
:10563000637AF90E9307F00F63F42701130A8000D1
:10564000B3574901B38AFA0003C70A0013050002E1
:10565000B384294133074701330AE540E30E0AEAE0
:1056600033194901B3DAE900B395490133D7EC00A6
:1056700093540901336BB70013850A009385040026
:10568000EF0080369309050093850400931B090100
:1056900013850A00EF00C03093DB0B019305050072
:1056A00013850B00EF00002D9399090193570B010F
:1056B000B3E7F90033944C0163FAA700B3872701DD
:1056C00063E6270163F4A700B3872701B38AA740E5
:1056D0009385040013850A00EF000031930905004B
:1056E0009385040013850A00EF00802B93050500C5
:1056F00013850B00EF00002893150B019399090106
:1057000093D50501B3E5B90063FAA500B38525017A
:1057100063E6250163F4A500B3852501B384A540A4
:105720006FF09FDFB7070001130A0001E36AF9F089
:10573000130A80016FF0DFF0E3E8D5E8B707010056
:1057400063FCF604930BF00F33B5DB001315350043
:1057500033D7A60097B701009387C7ADB387E7009B
:1057600083CB070093050002B38BAB00338B7541ED
:10577000631E0B0263E4360163EACC003384CC4041
:10578000B386D94033B58C00B384A640130504001A
:10579000938504006FF05FE3B70700011305000174
:1057A000E3E8F6FA130580016FF09FFAB3966601FD
:1057B000335D7601336DDD0033D47901B395690132
:1057C00033DC7C0193540D01336CBC0013050400E1
:1057D00093850400B31A6601EF000021130A050047
:1057E000938504001305040033996C01931C0D018B
:1057F000EF00001B93DC0C0113040500930505006A
:1058000013850C00EF000017131A0A0113570C013F
:105810003367EA00130A0400637EA7003307A70179
:10582000130AF4FF6368A7016376A700130AE4FF75
:105830003307A701B309A740938504001385090026
:10584000EF00801A938504001304050013850900F6
:10585000EF000015930505009304050013850C0067
:10586000EF00401193150C011314040193D50501A9
:10587000B365B4001387040063FEA500B385A501DA
:105880001387F4FF63E8A50163F6A5001387E4FF1F
:10589000B385A501131A0A01B70C0100336AEA00A7
:1058A0001384FCFFB3778A0033F48A00B384A540E5
:1058B00013850700930504002326F100135A0A01FB
:1058C000EF00400B930905009305040013050A003F
:1058D000EF00400A13DC0A01930D050093050C004C
:1058E00013050A00EF0000098327C100130A050011
:1058F00093050C0013850700EF00C0073305B501C1
:1059000013D709013307A7006374B701330A9A015B
:10591000B70701009387F7FF935507013377F70027
:1059200013170701B3F7F900B3854501B307F70073
:1059300063E6B400639EB400637CF900338657418C
:10594000B3B7C700B385A541B385F54093070600FB
:10595000B307F9403339F900B385B440B385254125
:1059600033947501B3D767013365F400B3D565018E
:105970006FF09FC5130605001305000093F6150090
:10598000638406003305C50093D515001316160071
:10599000E39605FE678000006340050663C60506C2
:1059A00013860500930505001305F0FF630C06023E
:1059B00093061000637AB6006358C00013161600F1
:1059C00093961600E36AB6FE1305000063E6C50071
:1059D000B385C5403365D50093D61600135616001F
:1059E000E39606FE6780000093820000EFF05FFB05
:1059F00013850500678002003305A04063D80500C9
:105A0000B305B0406FF0DFF9B305B04093820000FA
:105A1000EFF01FF93305A040678002009382000079
:105A200063CA0500634C0500EFF09FF7138505007E
:105A300067800200B305B040E35805FE3305A0407F
:0C5A4000EFF01FF63305B0406780020055
:02000004800278
:1000000049444C4500000000482FFEFF102FFEFF22
:100010001E2FFEFF2C2FFEFF342FFEFF5830FEFF59
:100020002030FEFF2E30FEFF3C30FEFF4430FEFF4E
:10003000546D722053766300DC35FEFFDC35FEFF25
:10004000DC35FEFF5A36FEFF2A36FEFF5036FEFF35
:10005000DC35FEFFDC35FEFF5A36FEFF2A36FEFF9A
:10006000546D725100000000286E756C6C29000000
:10007000DE43FEFFDC45FEFFD245FEFFDC45FEFF12
:10008000DC45FEFFDC45FEFFDC45FEFF5C44FEFF79
:10009000DC45FEFFDC45FEFF1444FEFF6A44FEFF24
:1000A000DC45FEFF1E44FEFF2844FEFF2844FEFF01
:1000B0002844FEFF2844FEFF2844FEFF2844FEFF9C
:1000C0002844FEFF2844FEFF2844FEFFDC45FEFFD7
:1000D000DC45FEFFDC45FEFFDC45FEFFDC45FEFFA8
:1000E000DC45FEFFDC45FEFFDC45FEFFDC45FEFF98
:1000F000DC45FEFFDC45FEFFDC45FEFFDC45FEFF88
:10010000DC45FEFFDC45FEFFDC45FEFFDC45FEFF77
:10011000DC45FEFFDC45FEFFDC45FEFFDC45FEFF67
:10012000DC45FEFFDC45FEFFDC45FEFFDC45FEFF57
:10013000DC45FEFFDC45FEFFDC45FEFFDC45FEFF47
:10014000DC45FEFFDC45FEFFDC45FEFFDC45FEFF37
:10015000DC45FEFFDC45FEFFDC45FEFFDC45FEFF27
:10016000DC45FEFFDC45FEFFDC45FEFFDC45FEFF17
:100170008E44FEFF3A45FEFFDC45FEFFDC45FEFFF8
:10018000DC45FEFFDC45FEFFDC45FEFFDC45FEFFF7
:10019000DC45FEFF8644FEFFDC45FEFFDC45FEFF3E
:1001A0008E45FEFF9445FEFFDC45FEFFDC45FEFF6D
:1001B000A244FEFFDC45FEFF8845FEFFDC45FEFF56
:1001C000DC45FEFFAC45FEFF6D69616F750A0000FE
:1001D0006D69616F75320A0068756E6772790A0021
:1001E0004572726F7220696E207265636D757465F9
:1001F00078207461736B73200D0A00004368656397
:100200006B54696D6572000052656375727369762F
:10021000655F4D75746578005265633100000000BC
:100220005265633200000000526563330000000035
:10023000000102020303030304040404040404048D
:10024000050505050505050505050505050505055E
:10025000060606060606060606060606060606063E
:10026000060606060606060606060606060606062E
:10027000070707070707070707070707070707070E
:1002800007070707070707070707070707070707FE
:1002900007070707070707070707070707070707EE
:1002A00007070707070707070707070707070707DE
:1002B00008080808080808080808080808080808BE
:1002C00008080808080808080808080808080808AE
:1002D000080808080808080808080808080808089E
:1002E000080808080808080808080808080808088E
:1002F000080808080808080808080808080808087E
:10030000080808080808080808080808080808086D
:10031000080808080808080808080808080808085D
:10032000080808080808080808080808080808084D
:100330001000000000000000017A5200017C010161
:100340001B0D02004C000000180000004C4BFEFF8B
:10035000DC05000000440E30708903950781018898
:100360000292049305940696089709980A990B9AA5
:100370000C0370020AC144C844C944D244D344D4D3
:1003800044D544D644D744D844D944DA440E004432
:100390000B0000005000000068000000D850FEFF75
:1003A0000005000000440E507488028903930599EB
:1003B0000B810192049406950796089709980A9A6A
:1003C0000C9B0D0320010AC144C844C944D244D344
:1003D00044D444D544D644D744D844D944DA44DB41
:0803E000440E00440B00000074
:1003F400AAAAAAAA08000000FC8F010009000000B4
:040000058000004037
:00000001FF
